:02000000804E30
:100050007590FF75B0FFC2B5C2B2C2AF7589207589
:100060008DFD858D8B759850D28E31A9740AC398F9
:1000700050F8B8430F31A9B830F0784331B1783037
:1000800031B180E6B8492931A9B83010D2B3C2B233
:10009000D297D2B4C2B531B9C2B3800AD2B3C2B218
:1000A000D297D2B4C2B5784931B1783031B180BA83
:1000B000B8574831A9D2B2D297D2B4C2B5C2B3317F
:1000C000DC13D2B74002C2B7D2E7F59031D3C2B445
:1000D00000000000D2B431B931B9C2B27590FFD27C
:1000E000B7E59023D2E030B702C2E0D2B5F8C2B58E
:1000F00031DC785731B1F831B1016AB8565331A9C2
:10010000B83008780431B1D8FC016A740AC3984049
:100110003ED2B3C2B2D297D2B4C2B531CAC2B331A1
:10012000B9A900785631B17A047B007590FFD2B737
:100130007590FFD2B7E59023D2E020B702C2E0F875
:10014000D2B531DCC2B5F831B1DBE0DADCD9D801A7
:100150006AB8453731A9B830F6C2B2C297C2B5C243
:10016000B3792031B9D9FCC2B4791531B9D9FCD2EF
:0F017000B4791531B9D9FCC2B2D297C2B531B941
:10017F00D2B3784531B1783031B1016AB858C13155
:10018F00A9B830BCC2B5000000D2B5000000C2B59E
:10019F00785831B1783031B1016A3098FDC298A8E2
:1001AF00992288993099FDC29922C001C0027A0222
:1001BF007900D9FEDAFAD002D00122C0017900D934
:1001CF00FED00122C0017918D9FED00122C00179D9
:0A01DF0008C833C813D9FAD0012272
:00000001FF
